:100000000C9483010C94AB010C94AB010C949515EA
:100010000C9495150C9495150C94AB010C94AB01B4
:100020000C94AB010C94AB010C94AB010C94AB01A0
:100030000C94AB010C94AB010C94AB010C94AB0190
:100040000C944B150C94AB010C9419150C94F314EF
:100050000C94AB010C94AB010C94AB010C94AB0170
:100060000C94AB010C94AB0108000000BE92244933
:10007000123EABAAAA2ABECDCCCC4C3E00000080DA
:10008000BEABAAAAAA3E00000000BF000000803F4D
:100090000000000000084178D3BB4387D1133D190D
:1000A0000E3CC3BD4282AD2B3E68EC8276BED98F3A
:1000B000E1A93E4C80EFFFBE01C4FF7F3F0000007E
:1000C000000000407A10F35A00A0724E1809001088
:1000D000A5D4E80000E87648170000E40B540200BD
:1000E00000CA9A3B000000E1F505000080969800E8
:1000F000000040420F000000A08601000000102711
:1001000000000000E80300000000640000000000A0
:100110000A00000000000100000000002C76D888D2
:10012000DC674F0823DFC1DFAE59E1B1B796E5E3E5
:10013000E453C63AE651997696E8E6C28426EB89FE
:100140008C9B62ED407C6FFCEFBC9C9F40F2BAA59B
:100150006FA5F490055A2AF75C936B6CF9676DC133
:100160001BFCE0E40D47FEF520E6B500D0ED902E37
:100170000300943577050080841E080000204E0A95
:10018000000000C80C333333330F986E12831141D3
:10019000EF8D2114893BE65516CFFEE6DB18D1849E
:1001A0004B381BF77C1D901DA4BBE42420328472C5
:1001B0005E228100C9F124ECA1E53D27415454455C
:1001C0004E54452047505300636C696D3A00686592
:1001D0007572652F74657874653D00646174653D62
:1001E0000030310030310030310030300074726145
:1001F0006D653D00524D4300436C696D0044617470
:1002000065486575726500426967436C6F636B0092
:1002100048657572654869766572004865757265EE
:1002200045746500446562756700416E6E756C6566
:1002300072006E6F75766561753D00546578746502
:100240000056657273696F6E005265696E6974005D
:10025000526573657400636F6D6D616E64653D001A
:100260000000000800020100000304070000000075
:100270000000000000000000240027002A00434185
:100280004E20536869656C6420696E697469616C9D
:100290006973C3A90065727265757220696E6974AD
:1002A0002E2043414E20536869656C642C20726592
:1002B000636F6D6D656E63652064616E73203220BF
:1002C0007365632E00000000002300260029000053
:1002D000000000250028002B00040404040404048A
:1002E00004020202020202030303030303010204E5
:1002F00008102040800102040810200102040810A8
:10030000200058160C1A11241FBECFEFD8E0DEBF14
:10031000CDBF24E0A4EFB2E001C01D92AE3AB20717
:10032000E1F712E0A0E0B1E0ECE0F6E402C00590F5
:100330000D92A43FB107D9F711E0C2E8D1E004C0A3
:100340002197FE010E94D320C138D107C9F70E942E
:100350009E170C94F9220C9400008CBD9DBD08954D
:10036000FC01248135816217730720F4808191811B
:10037000009729F41092590389E593E00895860FB8
:10038000971F08950895CF93DF93EC012FB7F8944A
:100390008091550390915603A0915703B091580353
:1003A0002FBF88879987AA87BB87E881F981028454
:1003B000F385E02DCE01099597FF1EC02FB7F89465
:1003C0008091550390915603A0915703B091580323
:1003D0002FBF488559856A857B85841B950BA60BA5
:1003E000B70B4C815D816E817F8184179507A607CD
:1003F000B707D8F28FEF9FEFDF91CF910895AF92BB
:10040000BF92CF92DF92EF92FF920F931F93CF9301
:10041000DF936C017B018B01040F151FEB015E0163
:10042000AE18BF08C017D10759F06991D601ED91F8
:10043000FC910190F081E02DC6010995892B79F797
:10044000C501DF91CF911F910F91FF90EF90DF9049
:10045000CF90BF90AF900895FC01538D448D252F10
:1004600030E0842F90E0821B930B541710F0CF964E
:10047000089501970895FC01918D828D981761F080
:10048000A28DAE0FBF2FB11D5D968C91928D9F5F97
:100490009F73928F90E008958FEF9FEF0895FC0176
:1004A000918D828D981731F0828DE80FF11D858D29
:1004B00090E008958FEF9FEF0895FC01918D228DBC
:1004C000892F90E0805C9F4F821B91098F73992741
:1004D000089585E693E00E945D0221E0892B09F4EE
:1004E00020E0822F089580E090E0892B29F00E947F
:1004F000690281110C9400000895FC01A48DA80FDD
:10050000B92FB11DA35ABF4F2C91848D90E0019655
:100510008F739927848FA689B7892C93A089B18975
:100520008C91837080648C93938D848D981306C016
:100530000288F389E02D80818F7D80830895EF927A
:10054000FF920F931F93CF93DF93EC0181E0888F8D
:100550009B8D8C8D98131AC0E889F989808185FF5D
:1005600015C09FB7F894EE89FF896083E889F989FF
:1005700080818370806480839FBF81E090E0DF9101
:10058000CF911F910F91FF90EF900895F62E0B8D54
:1005900010E00F5F1F4F0F731127E02E8C8D8E110F
:1005A0000CC00FB607FCFACFE889F989808185FF76
:1005B000F5CFCE010E947D02F1CFEB8DEC0FFD2F28
:1005C000F11DE35AFF4FF0829FB7F8940B8FEA8931
:1005D000FB8980818062CFCF0F931F93CF93DF93EE
:1005E0008C01D0E0C0E0F801EC0FFD1F64916623A0
:1005F00041F085E693E00E949F02892B11F021963D
:10060000F2CFCE01DF91CF911F910F910895CF933B
:10061000DF93EC01888D8823B9F0AA89BB89E8892A
:10062000F9898C9185FD03C0808186FD0DC00FB6D0
:1006300007FCF7CF8C9185FFF2CF808185FFEDCF4E
:10064000CE010E947D02E9CFDF91CF91089590E025
:10065000FC01E05AFD4F2491FC01E351FD4F349120
:10066000FC01E752FD4FE491EE23C9F0222339F05B
:10067000233001F1A8F4213019F1223029F1F0E002
:10068000EE0FFF1FE153FD4FA591B4918FB7F89482
:10069000EC91611126C030953E233C938FBF0895A5
:1006A0002730A9F02830C9F0243049F78091800024
:1006B0008F7D03C0809180008F7780938000DFCF93
:1006C00084B58F7784BDDBCF84B58F7DFBCF8091E0
:1006D000B0008F778093B000D2CF8091B0008F7D33
:1006E000F9CF3E2BDACFCF93DF9390E0FC01E351BB
:1006F000FD4F249187529D4FFC0184918823D1F0B6
:1007000090E0880F991FFC01EC58FD4FA591B49122
:10071000FC01E153FD4FC591D49161110EC09FB70B
:10072000F8948C91E22FE0958E238C932881E2231C
:10073000E8839FBFDF91CF9108958FB7F894EC9134
:10074000E22BEC938FBFF6CF3FB7F8948091510323
:1007500090915203A0915303B091540326B5A89BE6
:1007600005C02F3F19F00196A11DB11D3FBFBA2F43
:10077000A92F982F8827BC01CD01620F711D811D03
:10078000911D42E0660F771F881F991F4A95D1F788
:1007900008958F929F92AF92BF92CF92DF92EF9285
:1007A000FF924B015C010E94A4036B017C010E943B
:1007B000A4036C197D098E099F09683E7340810569
:1007C0009105A8F321E0821A9108A108B10888EEEA
:1007D000C80E83E0D81EE11CF11C81149104A10411
:1007E000B10429F7FF90EF90DF90CF90BF90AF90CA
:1007F0009F908F90089520915C0330915D0328179E
:10080000390771F490915A0380915B03981741F076
:10081000E0915A03F0E0E05FFC4F808190E00895A2
:100820008FEF9FEF08950895EF92FF920F931F931C
:10083000CF93DF93DC015C96ED90FC905D97E11423
:10084000F10479F481E090E013969C938E931297D3
:1008500090E080E0DF91CF911F910F91FF90EF909A
:1008600008955196ED91FC91529750968C91509726
:10087000982F90950FB75E962C915E97122F12705D
:1008800021FD6095F8942081112319F1282B2083F4
:10089000E7012197F1F728E0462F50E0308160FF13
:1008A0001AC0382B3083E7012197F1F7BA0175950B
:1008B0006795215089F7112381F0808189238083F6
:1008C0000FBF5C968D919C910197F1F781E090E0CC
:1008D000C1CF2923DCCF3923E5CF9081892BEFCFFE
:1008E00020915C0330915D032817390771F48091E2
:1008F0005B0320915A0390E0805C9F4F821B91091B
:1009000060E470E00E946A20089590E080E008951D
:1009100020915C0330915D0328173907B9F4909159
:100920005A0380915B03981789F0E0915A03F0E035
:10093000E05FFC4F808120915A0330E02F5F3F4FF2
:100940002F73332720935A0390E008958FEF9FEF82
:10095000089590E080E0089508958EBD00000DB4E4
:1009600007FEFDCF8EB508951F93CF93DF93182F09
:1009700080E591E00E94AD01C2E2D4E060E08E81AA
:100980000E94270383E00E94AD04812F0E94AD04E2
:1009900080E00E94AD04182F61E08E810E94270341
:1009A000812FDF91CF911F910895FF920F931F9395
:1009B000CF93DF93F82E062F142F80E591E00E944D
:1009C000AD01C2E2D4E060E08E810E94270385E0A1
:1009D0000E94AD048F2D0E94AD04802F0E94AD04B3
:1009E000812F0E94AD0461E08E81DF91CF911F9134
:1009F0000F91FF900C942703CF93C82F482F60EEE0
:100A00008FE00E94D5048FE00E94B404982F907E5E
:100A100081E09C1301C080E0CF9108951F93CF9394
:100A2000DF9380E591E00E94AD01C2E2D4E060E096
:100A30008E810E94270380EA0E94AD0480E00E941C
:100A4000AD04182F61E08E810E942703812FDF9172
:100A5000CF911F9108954F925F926F927F928F92E4
:100A60009F92AF92BF92CF92DF92EF92FF920F933D
:100A70001F93CF93DF9300D000D0CDB7DEB72B010B
:100A80003C016A01409223045092240460922504A0
:100A9000709226041092220410922704F12CE12C6B
:100AA00043E0A42EB12C53E2852E912C0E940E051A
:100AB00084758435C9F190912B04B501691B7109C6
:100AC00090E0292F30E02617370774F54FEF933069
:100AD00020F4F901EE56FE4F4081482319F510E548
:100AE000933020F4F901E157FE4F10811F5F60E061
:100AF000933020F424573E4FF901608140E08CE2AE
:100B00000E94D50480E0FFEFEF1AFF0A823079F4EB
:100B100082E3E816F10411F496E08FC0C401019756
:100B2000F1F7C4CF9F5FCDCF10E082E0ECCF92E32E
:100B3000E916F10489F302E4113439F004E41135C3
:100B400021F000E4113309F000E0C20123E09695A2
:100B500087952A95E1F789834294440C30EE43222D
:100B60004A821C821B8280E591E00E94AD0160E018
:100B7000809128040E942703802F0E94AD04FE016B
:100B800031967F015E01F5E0AF0EB11CF701819156
:100B90007F010E94AD04AE14BF04C1F788E00E943B
:100BA000AD04F12CE12CF601EE0DFF1D80810E94B9
:100BB000AD04FFEFEF1AFF0A88E0E816F10499F799
:100BC00061E0809128040E94270380E591E00E9463
:100BD000AD0160E0809128040E94270382E811346F
:100BE00039F084E8113521F081E8113309F080E013
:100BF0000E94AD0461E0809128040E942703F12C3B
:100C0000E12C115083E2C82ED12C9FEFE91AF90A8A
:100C1000812F0E94B404982F987083FF0AC0E2E3EA
:100C2000EE16F10411F497E008C0C6010197F1F740
:100C3000ECCFF2E3EF16F104B1F3892F0F900F9090
:100C40000F900F90DF91CF911F910F91FF90EF9038
:100C5000DF90CF90BF90AF909F908F907F906F90DC
:100C60005F904F9008950F931F93CF93DF93082FBA
:100C7000162F80E591E00E94AD01C2E2D4E060E071
:100C80008E810E94270382E00E94AD04802F0E9483
:100C9000AD04812F0E94AD0461E08E81DF91CF9180
:100CA0001F910F910C9427034F925F926F927F9246
:100CB0008F929F92AF92BF92CF92DF92EF92FF926C
:100CC0000F931F93CF93DF9300D000D0CDB7DEB743
:100CD000B82E6B013A01290160E0809128040E943E
:100CE00027038B2D0E94AD04CE0101965C014E01BD
:100CF00095E0890E911C80E00E94AD04F50181937E
:100D00005F01E815F905B9F72A818981F8E08F9F1D
:100D1000C0011124422F50E065E0559547956A9532
:100D2000E1F7840F951F092E000CAA0BBB0BF601EF
:100D300080839183A283B383F301108223FF3AC09F
:100D4000F60180819181A281B38132E0880F991FE1
:100D5000AA1FBB1F3A95D1F72370820F911DA11DC9
:100D6000B11D80839183A283B38380819181A2810D
:100D7000B381BA2FA92F982F88272B81820F911D1D
:100D8000A11DB11D80839183A283B3838081918152
:100D9000A281B381BA2FA92F982F88272C81820F87
:100DA000911DA11DB11D80839183A283B38381E036
:100DB000F301808380E00E94AD04982F9F70F801BA
:100DC000908386FB882780F9F2018083D12CC12C87
:100DD000F8018081C81680F4F8E0CF16D10461F0E4
:100DE0005701AC0CBD1C80E00E94AD04F50180836E
:100DF000FFEFCF1ADF0AECCF61E0809128040F905B
:100E00000F900F900F90DF91CF911F910F91FF9056
:100E1000EF90DF90CF90BF90AF909F908F907F909A
:100E20006F905F904F900C942703CF93C82F90E062
:100E300080E00E94721EC81731F06C2F90E080E0B5
:100E4000CF910C947A1ECF910895FC01019000205F
:100E5000E9F73197AF01481B590BBC0185E693E0D8
:100E60000C94FF0142E050E062EA72E085E693E014
:100E70000C94FF01CF93DF930E94EC02EC010E94DF
:100E800032078C0F9D1FDF91CF91089580916403ED
:100E9000882321F08CEB91E00E943A074EE551E067
:100EA00066E070E080E090E00E942B0540E551E0B4
:100EB00060E874E080E090E00E942B0548E051E09B
:100EC00060E874E080E090E00E942B0540E051E093
:100ED00060E874E080E090E00E942B0548E351E078
:100EE00060E874E080E090E00E942B0540E351E070
:100EF00060E874E080E090E00E942B0548E251E059
:100F000060E874E080E090E00E942B0540E251E050
:100F100060E874E080E090E00E942B0548E151E039
:100F200060E874E080E090E00E942B0540E151E031
:100F300060E874E080E090E00C942B05CF93DF93A1
:100F4000FC01448155816081718185E693E00E94B6
:100F5000FF01EC010E9432078C0F9D1FDF91CF91A2
:100F60000895FC0180819181009711F00C94651A1D
:100F700060E070E0CB010895FC0124813581FB0124
:100F80004481558124173507E1F4FC01808191816A
:100F9000FB01608171810097D1F061157105A1F4A9
:100FA000232BC1F0FC01808190E008C0232B91F03D
:100FB000FB01808190E091958195910921E0892B39
:100FC00009F020E0822F08950E94CF22F7CF61150B
:100FD000710561F721E0F6CF0F931F93CF93DF9355
:100FE0008C01EB01FC01808191810097E1F0688127
:100FF000798161157105A9F0428153812C813D8170
:101000004217530770F00E94D8228C819D81F8010D
:10101000958384831D821C82DF91CF911F910F9154
:1010200008950E94752188819981F80191838083B8
:101030008A819B81938382838C819D819583848324
:10104000198218821B821A82E5CFCF93DF93EC01BD
:1010500088819981009711F00E9475211982188268
:101060001D821C821B821A82DF91CF910895FC01A0
:10107000808191810C9475210F931F93CF93DF93FF
:10108000EC0188819981009759F02A813B812617CC
:10109000370730F081E0DF91CF911F910F910895D4
:1010A0008B016F5F7F4F0E94FE21009759F099835B
:1010B00088831B830A832C813D81232B59F7FC01F4
:1010C0001082E8CF80E0E7CFEF92FF920F931F935B
:1010D000CF93DF936115710541F480E0DF91CF91EB
:1010E0001F910F91FF90EF90089541155105B1F0B8
:1010F0007B01EC010C811D81040F151FB8010E94BA
:101100003C08882351F3288139818C819D81B70166
:10111000820F931F0E94D8221D830C8381E0DECFB3
:10112000CF93DF93EC01FB01448155816081718194
:101130000E946408811103C0CE010E942508CE01DF
:10114000DF91CF910895EF92FF920F931F93CF936A
:10115000DF93EC018B01CB010E94931A7C01BC014F
:10116000CE010E943C0881110BC0CE010E942508CF
:10117000CE01DF91CF911F910F91FF90EF900895D5
:10118000FD82EC82B801888199810E948C1AF0CF8F
:10119000FC011182108213821282158214820C9437
:1011A000A308EF92FF920F931F93CF93DF93EC016D
:1011B0007B018A01BA010E943C0881110BC0CE015B
:1011C0000E942508CE01DF91CF911F910F91FF90D2
:1011D000EF9008951D830C83B701888199810E9447
:1011E000D822F0CFFB0101900020E9F73197AF0141
:1011F000461B570B0C94D1080F931F93CF93DF938B
:10120000CDB7DEB762970FB6F894DEBF0FBECDBF85
:101210008C01CB01F8011182108213821282158297
:1012200014824AE0BE016F5F7F4F0E949C1ABE018C
:101230006F5F7F4FC8010E94F20862960FB6F89464
:10124000DEBF0FBECDBFDF91CF911F910F910895EB
:101250000F931F93CF93DF93CDB7DEB729970FB6C8
:10126000F894DEBF0FBECDBF8C01862FF80111822E
:10127000108213821282158214824AE0BE016F5FCF
:101280007F4F90E00E94ED1ABE016F5F7F4FC80153
:101290000E94F20829960FB6F894DEBF0FBECDBFAC
:1012A000DF91CF911F910F910895EF92FF920F93CD
:1012B0001F93CF93DF93CDB7DEB7A1970FB6F89406
:1012C000DEBF0FBECDBF7C01CB01BA01F701118299
:1012D000108213821282158214828E010F5F1F4FBB
:1012E00022E044E00E94471A009789F0BC01C70140
:1012F0000E94F208A1960FB6F894DEBF0FBECDBFD4
:10130000DF91CF911F910F91FF90EF900895C7014A
:101310000E942508EFCFCF93DF93EC01FB018617E6
:10132000970749F0608171816115710541F0448131
:1013300055810E94D108CE01DF91CF9108950E947E
:101340002508F9CFFC0111821082138212821582C6
:101350001482FB0101900020E9F73197AF01461B91
:10136000570B0C94D108EF92FF920F931F93CF93DA
:10137000DF9300D0CDB7DEB78C017B0164EA72E069
:101380000E94A209C7010E94C30197FD0EC08A30C6
:10139000910559F089831A8241E050E0BE016F5FE8
:1013A0007F4FC8010E946408EDCFC8010F900F90D5
:1013B000DF91CF911F910F91FF90EF900895AF9221
:1013C000BF92CF92DF92EF92FF920F931F93CF9332
:1013D000DF936C015B017A0189012417350720F442
:1013E0008F2D7901042F182F64EA72E0C6010E9444
:1013F000A209D5011496CD91DC91EC16FD06E0F41E
:101400000C171D0708F4E801D501ED91FC91119727
:10141000EC0FFD1F108110826D917C916E0D7F1D70
:10142000C60161157105A1F00E94F208F5018081E5
:101430009181C80FD91F1883C601DF91CF911F91E9
:101440000F91FF90EF90DF90CF90BF90AF900895F5
:101450000E942508EBCF4F925F926F927F928F92FE
:101460009F92AF92BF92EF92FF920F931F93CF93F1
:10147000DF93CDB7DEB7CB54D1090FB6F894DEBFFA
:101480000FBECDBF85E693E00E945D02892B09F473
:10149000A3C265E673E0CE010F960E94B309809166
:1014A0006403882341F086E592E00E94EC02CE01BD
:1014B0000F960E949E0760E572E0CE0101960E94A1
:1014C000C808BE016F5F7F4FCE010F960E94BC0718
:1014D000182FCE0101960E943708112319F0F0E071
:1014E000E0E0099569E472E0CE0101960E94C80827
:1014F000BE016F5F7F4FCE010F960E94BC07182F71
:10150000CE0101960E943708112329F080E00E9445
:1015100015071092610361E472E0CE0101960E940A
:10152000C808BE016F5F7F4FCE010F960E94BC07B7
:10153000182FCE0101960E943708112321F084EA6A
:1015400094E00E949E076BE372E0CE0101960E9438
:10155000C808BE016F5F7F4FCE010F960E94BC0787
:10156000182FCE0101960E943708112309F47CC080
:1015700064EA72E0CE0101960E94A20985E693E03A
:101580000E945D02892B89F065E673E0CE01099621
:101590000E94B309BE01675F7F4FCE0101960E9492
:1015A000EC07CE0109960E9437088D819E81892B18
:1015B00029F3E981FA818081882301F32CE030E06E
:1015C00050E040E0BE016F5F7F4FCE0109960E9460
:1015D000DF09BE01675F7F4FCE0101960E94EC07D5
:1015E000CE0109960E94370880916403882341F058
:1015F00082E392E00E94EC02CE0101960E949E07D7
:101600006AE272E0CE0109960E94C808BE01675FD7
:101610007F4FCE0101960E94BC07182FCE0109967C
:101620000E94370811111CC064E272E0CE010996D5
:101630000E94C808BE01675F7F4FCE0101960E94DD
:10164000BC07182FCE0109960E943708112309F410
:1016500034C380916403882309F42BC3109264037C
:10166000CE0101960E9437086BE172E0CE0101962F
:101670000E94C808BE016F5F7F4FCE010F960E9487
:10168000BC07182FCE0101960E943708112329F0BC
:10169000809161038B7F8093610360E172E0CE01F2
:1016A00001960E94C808BE016F5F7F4FCE010F9662
:1016B0000E94BC07182FCE0101960E943708112303
:1016C00029F08091610384608093610367E072E098
:1016D000CE0101960E94C808BE016F5F7F4FCE0108
:1016E0000F960E94BC07182FCE0101960E94370862
:1016F000112389F081E080935E014EE551E066E0C0
:1017000070E080E090E00E942B05809161038D7F66
:101710008160809361036DEF71E0CE0101960E94BC
:10172000C808BE016F5F7F4FCE010F960E94BC07B5
:10173000182FCE0101960E943708112381F082EA0A
:1017400080935E014EE551E066E070E080E090E05D
:101750000E942B05809161038C7F8093610368EF69
:1017600071E0CE0101960E94C808BE016F5F7F4FF5
:10177000CE010F960E94BC07182FCE0101960E9441
:101780003708112309F41AC120E030E040EA51E49F
:1017900060910C0370910D0380910E0390910F03E3
:1017A0000E94C01E0E949E1FCE0109960E94FC0846
:1017B00069EB71E0CE0101960E94A209BE01675F4C
:1017C0007F4FCE0101960E9490080E949E07CE0195
:1017D00001960E943708CE0109960E94370868ECEE
:1017E00070E080E090E00E94C90320E030E040E03B
:1017F0005FE3609108037091090380910A0390915F
:101800000B030E94B41D20E030E048E851E40E9440
:10181000C01EAB01BC01CE0109960E9455096CEBBC
:1018200071E0CE0101960E94A209BE01675F7F4F61
:10183000CE0101960E9490080E949E07CE0101965B
:101840000E943708CE0109960E94370868EC70E0C4
:1018500080E090E00E94C90360915D01CE0109968D
:101860000E9428096FEB71E0CE0101960E94A20947
:10187000BE01675F7F4FCE0101960E9490080E94D3
:101880009E07CE0101960E943708CE0109960E945C
:10189000370868EC70E080E090E00E94C903609136
:1018A0005C01CE0109960E94280962EC71E0CE012C
:1018B00001960E94A209BE01675F7F4FCE0101968B
:1018C0000E9490080E949E07CE0101960E94370850
:1018D000CE0109960E94370868EC70E080E090E045
:1018E0000E94C90360915B01CE0109960E942809FC
:1018F00065EC71E0CE0101960E94A209BE01675F0E
:101900007F4FCE0101960E9490080E949E07CE0153
:1019100001960E943708CE0109960E94370868ECAC
:1019200070E080E090E00E94C90380915A0164E178
:101930000E945E20E82FE150FF0BBF01CE01099607
:101940000E94FC0868EC71E0CE0101960E94A20999
:10195000BE01675F7F4FCE0101960E9490080E94F2
:101960009E07CE0101960E943708CE0109960E947B
:10197000370868EC70E080E090E00E94C903609155
:1019800059016150770BCE0109960E94FC086BEC5F
:1019900071E0CE0101960E94A209BE01675F7F4FF0
:1019A000CE0101960E9490080E949E07CE010196EA
:1019B0000E943708CE0109960E9437088091610382
:1019C0000E94150764EA72E0CE010F960E94F208A9
:1019D000CE010F960E94370864EA72E0CE01459668
:1019E0000E94A20964EA72E0CE014B960E94A2090D
:1019F00064EA72E0CE0181960E94A20964EA72E074
:101A0000CE0187960E94A20964EA72E0CE018D960B
:101A10000E94A20964EA72E0CE01C3960E94A20964
:101A200064EA72E0CE01C9960E94A20964EA72E0FB
:101A3000CE01CF960E94A20983E094E00E94700438
:101A4000892B09F47BC163E074E0CE0101960E940A
:101A5000B309BE016F5F7F4FCE0145960E94EC0730
:101A6000CE0101960E94370864EF71E0CE01019625
:101A70000E94C808898D9A8D892B61F0ED88FE88B7
:101A800069817A81C7010E94DF228C010E191F092A
:101A9000892B11F40FEF1FEF1093600300935F0386
:101AA000CE0101960E94370817FDC7C480916403D8
:101AB000882369F18DEE91E00E94EC02898D9A8D68
:101AC0000817190770F4ED88FE886AE270E0C70114
:101AD000800F911F0E94C4229C012E193F09892B5F
:101AE00011F42FEF3FEF2D5F3F4FA80143505109F5
:101AF000BE016B5E7F4FCE0101960E94DF09CE01D1
:101B000001960E949E07CE0101960E943708E09040
:101B10005F03F0906003898D9A8DE816F90608F04E
:101B200005C10D891E896AE270E0C8018E0D9F1DF6
:101B30000E94C422009709F4F9C09C01201B310BBC
:101B4000890158013AE0A31AB108380188E0681AFF
:101B500071089301A501BE016B5E7F4FCE01019616
:101B60000E94DF09BE016F5F7F4FCE0181960E9408
:101B7000EC07CE0101960E943708480196E0891AC9
:101B800091089401A301BE016B5E7F4FCE010196C7
:101B90000E94DF09BE016F5F7F4FCE0187960E94D2
:101BA000EC07CE0101960E943708980124503109B4
:101BB000A401BE016B5E7F4FCE0101960E94DF093A
:101BC000BE016F5F7F4FCE018D960E94EC07CE0164
:101BD00001960E943708CE0181960E94B10761509C
:101BE0007109810991096F3171058105910508F02D
:101BF000A0C0CE0187960E94B1076150710981098A
:101C000091096C3071058105910508F092C0CE01F3
:101C10008D960E94B1076351710981099109603560
:101C200071058105910508F084C010925801970153
:101C30002A5F3F4FA7014C5F5F4FBE016B5E7F4F36
:101C4000CE0101960E94DF09BE016F5F7F4FCE017A
:101C5000C3960E94EC07CE0101960E94370880913E
:101C6000610382FD6EC0CE01C3960E94B107AB0135
:101C7000BC014E5F5F4F6F4F7F4FCE0101960E94B8
:101C80002B16BE016F5F7F4FCE01C3960E94EC07FB
:101C9000CE0101960E943708CE01C3960E94B1077B
:101CA000693171058105910509F0CEC067EE71E0DB
:101CB0006DC081E080936403D3CCBE016F5F7F4F22
:101CC0008CE294E00E948B091092600310925F03F3
:101CD00000915F03109160030C301105ACF4B80162
:101CE0008CE294E00E94B001DC016C91C801019685
:101CF0000E947A1E80915F039091600301969093F9
:101D0000600380935F03E4CF82EA80935E014EE537
:101D100051E066E070E080E090E00E942B05809149
:101D200061038E7F8260809361039ACC0FEF1FEF77
:101D300008CF80915801882309F47FC30E94460789
:101D40007CC3CE01C3960E94B107AB01BC014F5FBB
:101D50005F4F6F4F7F4FCE0101960E942B16BE0141
:101D60006F5F7F4FCE01C3960E94EC07CE010196B4
:101D70000E943708CE01C3960E94B10768317105F1
:101D80008105910509F060C06AEE71E0CE01C3964D
:101D90000E94A308CE0181960E94B107AB01BC014D
:101DA0004F5F5F4F6F4F7F4FCE0101960E942B1602
:101DB000BE016F5F7F4FCE0181960E94EC07CE017E
:101DC00001960E943708CE0187960E94B1076630BF
:101DD00071058105910571F00CF002C26230710548
:101DE0008105910509F412C26430710581059105E0
:101DF00009F002C2CE0181960E94B1076F317105D0
:101E0000810591050CF40CC264EE71E0CE0181965F
:101E10000E94A308CE0187960E94B107AB01BC01C6
:101E20004F5F5F4F6F4F7F4FCE0101960E942B1681
:101E3000BE016F5F7F4FCE0187960E94EC07CE01F7
:101E400001960E943708ECC1AB20A09409F4A2CF00
:101E5000CE0187960E94B1072B013C016EE070E035
:101E600080E090E064197509860997092CE030E05C
:101E700040E050E00E947E204901CE018D960E94F4
:101E8000B1077B01E818F908CE0181960E94B107DD
:101E90001A8219821C821B821E821D8287010F2CCE
:101EA000000C220B330BAB01BC01400F511F621F12
:101EB000731F9701F7FE02C02D5F3F4F35952795A1
:101EC000359527958901330F220B330B040F151F0E
:101ED000261F371FC70164E670E00E946A20CB010D
:101EE000770FAA0BBB0B081B190B2A0B3B0BC70167
:101EF00060E971E00E946A20072E000C880B990BA4
:101F0000060F171F281F391F8CE0889DA001899D8F
:101F1000500D1124C2010297480F591F6FE1649FB1
:101F2000C001659F900D11246CE070E00E946A2052
:101F3000072E000C880B990B600F711F821F931FD7
:101F400027E030E040E050E00E947E2016E0169F3F
:101F50009001179F300D1124B90166587B4FCE01B7
:101F600001960E948B0960E2CE0101960E940D1637
:101F7000BE016F5D7F4F0E94900860E20E940D16C7
:101F8000B1E04B1A510861087108149DB001159D0C
:101F9000700D11246E5C7B4F0E9490088C0143E011
:101FA00050E06EEC71E00E946408811103C0C8012A
:101FB0000E942508BE01635D7F4FC8010E94900802
:101FC000BC01CE014B960E948B09CE0101960E9466
:101FD000370880916403882341F08BED91E00E94E3
:101FE000EC02CE014B960E949E074EE551E066E062
:101FF00070E080E090E00E942B0540E551E060E851
:1020000074E080E090E00E942B05A9E4EA2EA1E0B4
:10201000FA2E10E000E0B801CE014B960E94B0010C
:10202000FC018081D7018D937D010F5F1F4F073029
:10203000110589F748E451E060E874E080E090E041
:102040000E942B05F1E4EF2EF1E0FF2E07E010E0F7
:10205000B801CE014B960E94B001FC018081D701EE
:102060008D937D010F5F1F4F0E30110589F740E4FE
:1020700051E060E874E080E090E00E942B05E9E325
:10208000EE2EE1E0FE2EB801CE014B960E94B0018B
:10209000FC018081D7018D937D010F5F1F4F0531BA
:1020A000110589F748E351E060E874E080E090E0D2
:1020B0000E942B0571E3E72E71E0F72EB801CE01E7
:1020C0004B960E94B001FC018081D7018D937D0168
:1020D0000F5F1F4F0C31110589F740E351E060E8B5
:1020E00074E080E090E00E942B0548E251E060E857
:1020F00074E080E090E00E942B0540E251E060E84F
:1021000074E080E090E00E942B05CE01C3960E940F
:10211000B107062FE0905F03F09060035701B8E02D
:10212000AB0EB11CA7014A5F5F4F9501BE016B5E0C
:102130007F4FCE0101960E94DF09BE016F5F7F4F86
:10214000CE01C9960E94EC07CE0101960E94370885
:10215000CE01C9960E94B107162F9701265F3F4F07
:10216000A501BE016B5E7F4FCE0101960E94DF0983
:10217000BE016F5F7F4FCE01CF960E94EC07CE016C
:1021800001960E943708CE01CF960E94B107809138
:10219000610381FF6FC06CE274E0CE0145960E943E
:1021A0008B091092600310925F0360E2B62EE090FC
:1021B0005F03F09060038F8D98A1E816F90608F090
:1021C00085C0B701CE014B960E94B001FC01B082E0
:1021D000FFEFEF1AFF0AF0926003E0925F03E7CF90
:1021E000693071058105910509F404CE6B307105E4
:1021F0008105910509F4FECDCE0181960E94B107BB
:1022000060327105810591055CF0FECDCE018196AD
:102210000E94B1076D317105810591050CF0F4CD77
:10222000CE0187960E94B1076D3071058105910539
:102230000CF40ECE61EE71E0CE0187960E94A308E9
:10224000CE018D960E94B107AB01BC014F5F5F4F7D
:102250006F4F7F4FCE0101960E942B16BE016F5F1C
:102260007F4FCE018D960E94EC07CE0101960E9411
:102270003708EECD1A8219821C821B821E821D82B3
:1022800060FF1BC0BE016D5C7F4FCE0101960E94B6
:102290008B096AE3CE0101960E940D16BE01675CB0
:1022A0007F4F0E949008BC01CE0145960E948B0989
:1022B000CE0101960E94370874CFBE016D5C7F4F3E
:1022C000CE0101960E948B0960E2E4CF898D9A8D40
:1022D0006CE070E0681B790B7695679590E080E084
:1022E0000E94531D20E030E040E05FE30E94C01EEA
:1022F0000E949E1F7B017093600360935F03A09018
:102300005F03B0906003B5016E197F09898D9A8DC6
:1023100068177907B0F4CE0145960E94B0014C01D0
:10232000B501CE014B960E94B001D4012C91FC0165
:102330002083FFEFAF1ABF0AB0926003A0925F0341
:10234000DECF80916403882341F08EEC91E00E94FF
:10235000EC02CE014B960E949E0783E090E09093A2
:10236000600380935F03E0905F03F090600328E0D8
:10237000E216F104ACF4B70163507109CE014B963B
:102380000E94B001F701E85EFE4FDC018C91808372
:10239000BFEFEB1AFB0AF0926003E0925F03E3CF1A
:1023A00048E151E060E874E080E090E00E942B0595
:1023B00081E090E09093600380935F03E0905F037F
:1023C000F0906003E8E0EE16F104ACF4B7016C5F46
:1023D0007F4FCE014B960E94B001F701E05FFE4FA8
:1023E000DC018C918083BFEFEB1AFB0AF092600353
:1023F000E0925F03E3CF40E151E060E874E080E009
:1024000090E00E942B052AE0802F622F0E945E2020
:102410008295807F980F90930003812F0E945E2009
:102420008295807F980F9093010340E053E062E033
:1024300075E080E090E00E942B0580E480937C00B2
:1024400080917A00806480937A0080917A0086FD82
:10245000FCCF0091780060917900162F61E070E068
:1024600080E090E00E94C903B801110F880B990B1E
:102470000E94551D9B01AC0160E070EC8FE794E475
:102480000E942C1F20E030E040E85FE30E94BF1E66
:102490009B01AC0160E070E68AEE96E40E942C1F7E
:1024A0000E94E11F4B015C012DE239ED46EC53E344
:1024B0000E94B41DA50194010E94B41DA5019401C0
:1024C0000E94B41D2B013C0129E33CEB4FE659E38C
:1024D000C501B4010E94B41D25E739EC4AE65AE370
:1024E0000E94C01E9B01AC01C301B2010E94C01E2C
:1024F0009B01AC0160E070E080E89FE30E942C1F2C
:1025000023E333E948E853E40E94BF1E60930C03C1
:1025100070930D0380930E0390930F032091FC02A0
:102520003091FD024091FE025091FF020E94C01EB8
:102530004B015C018092FC029092FD02A092FE028F
:10254000B092FF0260916203709163036F5F7F4FEF
:1025500070936303609362036C3371050CF474C071
:10256000072E000C880B990B0E94551D9B01AC0196
:10257000C501B4010E942C1F4B015C0120E030E03A
:10258000A9010E94D41F20E030E040E05FE387FD16
:10259000F4C0C501B4010E94C01E0E949E1F0E948B
:1025A000551D4B015C018092FC029092FD02A092AD
:1025B000FE02B092FF0223EC35EF48EE5FE30E948B
:1025C000B41D20E030E042E952E40E94C01E0E94A7
:1025D0009E1F6093F50244EF52E061E075E080E0F9
:1025E00090E00E942B0520E030E040EA51E4C50174
:1025F000B4010E94C01E0E949E1FCE0109960E9437
:10260000FC0869EB71E0CE0101960E94A209BE01AF
:10261000675F7F4FCE0101960E9490080E949E073F
:10262000CE0101960E943708CE0109960E94370814
:102630001092FC021092FD021092FE021092FF0214
:1026400010926303109262032C961FAE2C9764EADB
:1026500072E0CE018B5B9F4F0E94A2090E940E0583
:10266000837009F44FC00E940E05982F9B7A292F82
:1026700030E095959595959590718370892BA9017A
:10268000559547954470842B359527953595279515
:102690002870822B80FF76C0FE0131967F018E016B
:1026A000055B1F4F27E234E042E254E063E274E04E
:1026B00080E90E9454068091230490912404813380
:1026C00031E0930709F473C08233914009F4C4C028
:1026D0002B968EAD9FAD2B97892BA1F02796EEAD53
:1026E000FFAD27978081882369F080916403882358
:1026F00049F088EC91E00E94EC02CE018B5B9F4F89
:102700000E949E07CE018B5B9F4F0E943708CE012F
:10271000CF960E943708CE01C9960E943708CE0195
:10272000C3960E943708CE018D960E943708CE01CD
:1027300087960E943708CE0181960E943708CE0105
:102740004B960E943708CE0145960E943708C55B1C
:10275000DF4F0FB6F894DEBF0FBECDBFDF91CF9134
:102760001F910F91FF90EF90BF90AF909F908F902F
:102770007F906F905F904F900895C501B4010E94C3
:10278000BF1E0BCF81FF0FC09E012F5F3F4F79010E
:102790008E01055B1F4F27E234E042E254E063E222
:1027A00074E084E986CF2C961FAE2C9784CF1A81D3
:1027B000612F70E090E080E00E94551D2091080399
:1027C0003091090340910A0350910B030E944E1D62
:1027D000882309F47DCF612F70E090E080E00E94B3
:1027E000531D609308037093090380930A03909329
:1027F0000B0320E030E040E05FE30E94B41D20E0E6
:1028000030E048E851E40E94C01EAB01BC01CE019B
:102810000F960E9455096CEB71E0CE0109960E945B
:10282000A209BE01615F7F4FCE0109960E94900808
:10283000BC01CE018B5B9F4F0E948B09CE01099694
:102840000E943708CE010F960E943708CE018B5B9D
:102850009F4F0E949E073CCF698180915D01681760
:1028600031F160935D01CE010F960E9428096FEB54
:1028700071E0CE0109960E94A209BE01615F7F4FFF
:10288000CE0109960E949008BC01CE018B5B9F4F40
:102890000E948B09CE0109960E943708CE010F963F
:1028A0000E943708CE018B5B9F4F0E949E076A8172
:1028B00080915C01681731F160935C01CE010F9645
:1028C0000E94280962EC71E0CE0109960E94A209DB
:1028D000BE01615F7F4FCE0109960E949008BC0146
:1028E000CE018B5B9F4F0E948B09CE0109960E94FF
:1028F0003708CE010F960E943708CE018B5B9F4FA1
:102900000E949E076B8180915B01681731F1609393
:102910005B01CE010F960E94280965EC71E0CE01A3
:1029200009960E94A209BE01615F7F4FCE01099600
:102930000E949008BC01CE018B5B9F4F0E948B09C7
:10294000CE0109960E943708CE010F960E943708E3
:10295000CE018B5B9F4F0E949E078C8190915A0104
:10296000891769F180935A0164E10E945E20E82F83
:10297000E150FF0BBF01CE010F960E94FC0868ECEE
:1029800071E0CE0109960E94A209BE01615F7F4FEE
:10299000CE0109960E949008BC01CE018B5B9F4F2F
:1029A0000E948B09CE0109960E943708CE010F962E
:1029B0000E943708CE018B5B9F4F0E949E0768855F
:1029C00080915901681709F483CE6A3008F080CEEF
:1029D000609359016150770BCE010F960E94FC085D
:1029E0006BEC71E01ACF1F920F920FB60F92112469
:1029F0002F933F934F935F936F937F938F939F9307
:102A0000AF93BF93EF93FF9385E693E00E947D021F
:102A1000FF91EF91BF91AF919F918F917F916F91B6
:102A20005F914F913F912F910F900FBE0F901F908C
:102A300018951F920F920FB60F9211242F938F9318
:102A40009F93EF93FF93E0917503F091760380815C
:102A5000E0917B03F0917C0382FD1BC0908180910B
:102A60007E038F5F8F7320917F03821741F0E09187
:102A70007E03F0E0EB59FC4F958F80937E03FF912E
:102A8000EF919F918F912F910F900FBE0F901F90FC
:102A900018958081F4CF1F920F920FB60F921124D8
:102AA0002F933F938F939F93AF93BF938091550341
:102AB00090915603A0915703B09158033091500361
:102AC00023E0230F2D3758F50196A11DB11D20934A
:102AD00050038093550390935603A0935703B093EC
:102AE00058038091510390915203A0915303B091E8
:102AF00054030196A11DB11D80935103909352037D
:102B0000A0935303B0935403BF91AF919F918F91C2
:102B10003F912F910F900FBE0F901F90189526E8B0
:102B2000230F0296A11DB11DD2CF1F920F920FB697
:102B30000F9211242F933F934F935F936F937F9343
:102B40008F939F93AF93BF93EF93FF93E0915C03B9
:102B5000F0915D03309749F0A685B7858585968D00
:102B600091FF14C09C918923A1F4FF91EF91BF9133
:102B7000AF919F918F917F916F915F914F913F9115
:102B80002F910F900FBE0F901F9018959C91892345
:102B900061F7A389B4899C918589809589238C9359
:102BA000868997890197F1F7608D718DA685B78524
:102BB000558538E020E0CB010197F1F7822F90E0B6
:102BC00095958795282F4C91452309F02068315021
:102BD00091F7868D81FD209580915B0390E00196B1
:102BE0008F73992730915A03381799F0A0915B039E
:102BF000B0E0A05FBC4F2C9380935B03828D938DDC
:102C00000197F1F7A389B4898C919589892B8C93CD
:102C1000ACCF868D8160868FF1CF0F931F93CF93BA
:102C2000DF9300D0CDB7DEB78C0169831A8241E013
:102C300050E0BE016F5F7F4F0E946408811103C0A6
:102C4000C8010E942508C8010F900F90DF91CF9115
:102C50001F910F9108950F931F93CF93DF93CDB7DB
:102C6000DEB7A2970FB6F894DEBF0FBECDBF8C01C2
:102C7000CB01BA01F80111821082138212821582EF
:102C800014822AE0AE014F5F5F4F0E94A71ABE0177
:102C90006F5F7F4FC8010E94F208A2960FB6F894AA
:102CA000DEBF0FBECDBFDF91CF911F910F91089571
:102CB000CF92DF92EF92FF92109268031092670317
:102CC00098EEC92E93E0D92EE12CF12CC092690325
:102CD000D0926A03E0926B03F0926C0389E991E071
:102CE000909366038093650385EC90E09093720364
:102CF0008093710384EC90E090937403809373034A
:102D000080EC90E0909376038093750381EC90E0E3
:102D1000909378038093770382EC90E090937A030A
:102D20008093790386EC90E090937C0380937B03FF
:102D300010927E0310927F03109280031092810301
:102D400062ED71E084EA94E00E94A20964EE71E011
:102D50008AE794E00E94A2096DEE71E080E894E0B9
:102D60000E94A20963EF71E086E894E00E94A20944
:102D700069EF71E08CE894E00E94A20962E072E0E1
:102D800082E994E00E94A20968E072E088E994E098
:102D90000E94A20961E172E08EE994E00E94A2091A
:102DA00068E172E082E394E00E94A20960E272E0CE
:102DB00088E394E00E94A20968E272E08EE394E066
:102DC0000E94A2096DE272E084E494E00E94A209EC
:102DD00063E372E08AE494E00E94A20967E372E090
:102DE00080E594E00E94A2096CE372E086E594E03D
:102DF0000E94A20964E472E08CE594E00E94A209BA
:102E000069E472E082E694E00E94A20963E572E060
:102E100088E694E00E94A2096BE572E08EE694E0F9
:102E20000E94A20964E672E084E794E00E94A2098D
:102E300064EA72E08CE294E00E94A20910922B04F2
:102E400082E094E090932A04809329048AE080939E
:102E5000280461E00E94730361E0809128040E94CD
:102E600027031092060410920504C0920704D09222
:102E70000804E0920904F0920A048BEA91E090932E
:102E800004048093030410921A04109219041092FF
:102E90001C0410921B0410921E0410921D04109228
:102EA000200410921F04609121046E7F6D7F609357
:102EB00021046695617081E0682784E00E94270301
:102EC00061E084E00E947303E1EFF2E0E491E093BB
:102ED0001304EDEDF2E0E491F0E0EE0FFF1FE1539B
:102EE000FD4F85919491909315048093140460E0B4
:102EF00083E00E9473038091210481FD04C061E09E
:102F000083E00E94270383E080930F04E0EFF2E068
:102F1000E491E0931004ECEDF2E0E491F0E0EE0FC8
:102F2000FF1FEB53FD4F8591949190931204809372
:102F30001104FF90EF90DF90CF900895CF93DF932F
:102F4000CDB7DEB72C970FB6F894DEBF0FBECDBF5E
:102F5000789484B5826084BD84B5816084BD85B574
:102F6000826085BD85B5816085BD80916E00816080
:102F700080936E0010928100809181008260809326
:102F80008100809181008160809381008091800028
:102F90008160809380008091B10084608093B10053
:102FA0008091B00081608093B00080917A0084604D
:102FB00080937A0080917A00826080937A00809179
:102FC0007A00816080937A0080917A008068809393
:102FD0007A001092C100E0917503F091760382E0CF
:102FE0008083E0917103F09172031082E09173038A
:102FF000F091740387E6808310927D03E09179035A
:10300000F0917A0386E08083E0917703F091780372
:10301000808180618083E0917703F09178038081E3
:1030200088608083E0917703F091780380818068E5
:103030008083E0917703F091780380818F7D808396
:1030400010921E0410921D0410921C0410921B0476
:1030500010921A04109219048DE991E090932004C3
:1030600080931F0490910F04963108F047C02DEB18
:1030700030E030931A04209319042BE931E03093A7
:103080001C0420931B042CE231E030931E04209397
:103090001D042091680084E0983048F031E09E30B3
:1030A00008F430E081E001C0880F3A95EAF7822BFE
:1030B000809368002DE630E0983050F02BE630E049
:1030C0009E3030F02CE630E0963110F030E020E019
:1030D0003093170420931604292F30E0983008F01D
:1030E000BFC081E001C0880F9A95EAF78093180469
:1030F00080911F04909120040197F1F780911D04A5
:1031000090911E04892B49F1E0915C03F0915D03DD
:1031100084E0E330F80709F1309739F0A389B489E6
:103120009C918589809589238C93809121048E7F41
:103130008093210410925B0310925A0383E094E081
:1031400090935D0380935C03E0911604F091170463
:10315000808190911804892B808361E08AE00E942D
:10316000730360E08AE00E94270393EEA92E92E0A9
:10317000B92E27EFE22E22E0F22EDFB6F8948091EE
:103180005E03811125C0F5018491F7019491E82F28
:10319000F0E0EE0FFF1FEC58FD4FA591B4918C911C
:1031A000982321F461E08AE00E94270361E08AE02D
:1031B0000E9473038CB580618CBD8CB580648CBD1E
:1031C00061E08DE00E94730361E08BE00E94730375
:1031D00080915E038F5F80935E03DFBE80E591E0A8
:1031E0000E94AD0160E0809128040E94270380ECDA
:1031F0000E94AD0461E0809128040E9427036AE0E8
:1032000070E080E090E00E94C90380E80E94FC0426
:10321000882399F18DE692E00E942507809164034E
:10322000882321F085E992E00E943A0760ED77E07B
:1032300080E090E00E94C903809162039091630353
:103240000196909363038093620305970CF495CFE6
:103250001092630310926203F0E0E0E009958DCFD5
:103260009E3040F42850310981E001C0880F2A9532
:10327000EAF73CCF2E503109F7CF87E892E00E9461
:10328000250761E08AE20E94330664EB89E20E942E
:10329000330666E088E20E94330685EA92E00E94E7
:1032A000250710E360E0812F0E94330660E080E193
:1032B000810F0E94330660E080E2810F0E94330696
:1032C0001F5F1E3379F760E080E60E94330660E0FE
:1032D00080E70E94330663E08BE20E94330644E0FD
:1032E00064E680E60E94D50440E060E680E70E9444
:1032F000D50480E00E94FC04882319F08AEB92E058
:103300008BCF85ED92E00E94250710926303109207
:10331000620380916403882321F08EE792E00E948B
:103320003A0760ED77E080E090E00E94C9034EE745
:1033300051E060E071E080E090E00E942B0546E7FC
:1033400051E066E070E080E090E00E942B054EE6E0
:1033500051E066E070E080E090E00E942B056AEFAB
:1033600070E080E090E00E94C90346E651E069E227
:1033700070E080E090E00E942B0590E080E00E94E9
:10338000721E182F8093610387FF11C080E00E9496
:10339000150700E010E00E942B0A01151105D9F372
:1033A0000E9469028823B9F30E940000F4CF81E0F3
:1033B00010FF82EA80935E014EE551E066E070E026
:1033C00080E090E00E942B0511FFE3CF1092600394
:1033D00010925F0300915F03109160030C301105A0
:1033E0009CF47801FFEFEF1AFF0AC7010E94721EDA
:1033F000E1E0F0E0EC0FFD1FE00FF11F8083F092A1
:103400006003E0925F03E6CFBE016F5F7F4F8CE207
:1034100094E00E94F208BDCFCF93DF938BEA91E056
:10342000909304048093030480915C0390915D0366
:103430008350944071F4E0911604F0911704908148
:103440008091180480958923808310925D031092E7
:103450005C038CE294E00E943708CAE7D4E0269728
:10346000CE010E94370884E0C233D807C1F7C4EA0E
:10347000D4E02697CE010E94370824E0CA37D2074D
:10348000C1F784EA94E0DF91CF910C943708EF9272
:103490000F931F93CF93DF93E80134E047FD34E1AE
:1034A000042E000C550B57FF03C05195419551094F
:1034B000E32E022F242FAE010E94071BCE01DF91C5
:1034C000CF911F910F91EF9008951F93FC019927C1
:1034D0008827BC01E89411911032E9F3193010F0FB
:1034E0001E30C8F31B3251F01D3249F4689406C0F7
:1034F0000E94B61A610F711D811D911D119110530B
:103500001A30B0F33EF490958095709561957F4F99
:103510008F4F9F4F1F910895FB01DC0105900D9285
:103520000020E1F70895FC0105900020E9F780955F
:1035300090958E0F9F1F0895BB274A3031F4992331
:1035400022F4BDE2909581959F4F0C94EE1ABB2713
:103550002A3051F4992342F4BDE2909580957095FC
:1035600061957F4F8F4F9F4F0C94CC1A592F482F46
:10357000372F262F660F771F881F991F660F771F1B
:10358000881F991F620F731F841F951F660F771F77
:10359000881F991F0895BB27FA01A62F621771058E
:1035A00081059105330B30FB66F0AA27660F771F64
:1035B000881F991FAA1FA21710F0A21B63953850ED
:1035C000A9F7A05DAA3308F0A95DA19336F7B11160
:1035D000B1931082CA010C943E1DBB27FB015527F5
:1035E000AA27880F991FAA1FA41710F0A41B839560
:1035F0005051B9F7A05DAA3308F0A95DA1930097D7
:1036000079F7B111B1931192CB010C943E1DA9E051
:10361000B0E0EDE0FBE10C948E1E6A01F22EB02EBC
:10362000102FFBE3AF2EA01608F41BE31F5F012F42
:1036300027E0AE014F5F5F4F0E94661CBC0189818D
:10364000982F9970913009F43FC09BE2E1FC04C0CF
:103650009E2D9170E0FC3AC05E2D5071E82FE8700D
:1036600083FF46C084E0911101C083E0EF2DE81B89
:103670008F1508F0E0E0D6018E2F20E2552351F19E
:10368000992329F0D6019C93C60101966C019601FD
:103690002D5F3F4FE2FE24C08EE4D6018C9391E46F
:1036A00011969C93119712968C93D9018E2F90E2CC
:1036B00081111BC0E20FF32FF11D10828EEF9FEFDF
:1036C0002996ECE00C94AA1E9DE2C6CF90E2C4CFEE
:1036D0002D9381508111FCCFCE0ED11CE0E0D0CFD4
:1036E0008EE6D6018C9391E6DBCF9D938150E0CF9F
:1036F000482F447082FF3DC084E0911101C083E0F7
:103700008F1510F4EF2DE81BD6018E2F20E25523E4
:1037100009F1992329F0D6019C93C60101966C0109
:1037200096012D5F3F4FE2FE1BC089E4D6018C93CA
:103730008EE411968C93119786E412968C93D9019E
:103740008E2F90E2882309F4B5CF9D938150FACF54
:103750002D9381508111FCCFCE0ED11CE0E0D9CF4A
:1037600089E6D6018C938EE611968C93119786E6A6
:10377000E4CF9B0177FF02C030E020E0A1E0B0E0A1
:10378000911102C0B0E0A0E0F9013196AE0FBF1F69
:103790008B2C912CBB2009F461C05401EFEFAE1AC1
:1037A000BE0AAA0DBB1DFA161B0619F014F04F2D08
:1037B0004A1B511188C0E3FC59C07601A42FB0E226
:1037C000A1114FC0C40ED11C992309F45BC040E085
:1037D000D6011196F60190836D01552309F448C076
:1037E000012F060F9A81582F507184FF03C0913327
:1037F00009F4015010160CF047C0093008F008E039
:10380000EEE2FE2E5B01A01AB1088501919481942D
:1038100091082F3F320729F4D601FC92F601319628
:103820006F016217730794F1021713077CF5DB0130
:10383000A21BB30BAA24A394B12CAC0EBD1EAA0DDF
:10384000BB1D11968C9121503109D6011196281576
:103850003905F4F0F60180836D01DBCFB12CA12C8A
:10386000A0CFF701B1937F01A150AACF9111B0CFA2
:10387000D601942F50E302C05D9391509111FCCF7B
:10388000C40ED11C40E0ACCF01E0BACF80E3DBCF67
:103890006217730731F4963388F4953311F4552386
:1038A00069F0F6018083FD01842F90E2811108C048
:1038B000A40FB11D1C9290E080E002CF81E3F1CF14
:1038C00091938150F3CF911183CF8ACF283008F0A4
:1038D00027E03327DA01990F311D87FD91600096AB
:1038E0006105710539F432602E5F3D9330E32A950E
:1038F000E1F708959F3F30F080387105610509F0C8
:103900003C5F3C5F3D93913008F08068911DDF93F0
:10391000CF931F930F93FF92EF92192F987F969555
:10392000E92F96959695E90FFF27E45EFE4F9927BC
:103930003327EE24FF24A701E7010590089407949C
:1039400028F4360FE71EF81E491F511D660F771F1A
:10395000881F991F0694A1F70590079428F4E70E95
:10396000F81E491F561FC11D770F881F991F661F1C
:103970000694A1F70590079428F4F80E491F561FE6
:10398000C71FD11D880F991F661F771F0694A1F7C7
:103990000590079420F4490F561FC71FD81F990F91
:1039A000661F771F881F0694A9F7849110951770DA
:1039B00041F0D695C79557954795F794E7941A9592
:1039C000C1F7E2ECF0E0689415901591359165919E
:1039D000959105907FE27395E118F10A430B560B20
:1039E000C90BD009C0F7E10CF11E431F561FC91FB8
:1039F000D01D7EF4703311F48A95E6CFE89401501F
:103A000030F0080F0AF40027021708F4202F23953E
:103A1000022F7A3328F079E37D932A95E9F710C0D5
:103A20007D932A9589F6069497956795379517950E
:103A30001794E118F10A430B560BC90BD00998F003
:103A400023957E9173957A3308F070E37C9320136D
:103A5000B8F77E9170617D9330F0839571E37D932B
:103A600070E32A95E1F71124EF90FF900F911F91D9
:103A7000CF91DF91992787FD90950895DC01FC0196
:103A8000672F71917723E1F7329704C07C916D9392
:103A900070836291AE17BF07C8F308950E94901D0E
:103AA00008F481E00895E89409C097FB3EF49095EE
:103AB0008095709561957F4F8F4F9F4F9923A9F007
:103AC000F92F96E9BB279395F69587957795679596
:103AD000B795F111F8CFFAF4BB0F11F460FF1BC0DA
:103AE0006F5F7F4F8F4F9F4F16C0882311F096E96D
:103AF00011C0772321F09EE8872F762F05C066231B
:103B000071F096E8862F70E060E02AF09A95660FD3
:103B1000771F881FDAF7880F9695879597F908958C
:103B2000990F0008550FAA0BE0E8FEEF16161706CE
:103B3000E807F907C0F012161306E407F50798F036
:103B4000621B730B840B950B39F40A2661F0232B4F
:103B5000242B252B21F408950A2609F4A140A695CB
:103B60008FEF811D811D08950E94C71D0C94381E82
:103B70000E942A1E38F00E94311E20F0952311F079
:103B80000C94211E0C94271E11240C946C1E0E9470
:103B9000491E70F3959FC1F3950F50E0551F629F2A
:103BA000F001729FBB27F00DB11D639FAA27F00D96
:103BB000B11DAA1F649F6627B00DA11D661F829FBD
:103BC0002227B00DA11D621F739FB00DA11D621FA2
:103BD000839FA00D611D221F749F3327A00D611DBF
:103BE000231F849F600D211D822F762F6A2F1124A1
:103BF0009F5750409AF0F1F088234AF0EE0FFF1FD4
:103C0000BB1F661F771F881F91505040A9F79E3F2A
:103C1000510580F00C94211E0C946C1E5F3FE4F360
:103C2000983ED4F3869577956795B795F795E79580
:103C30009F5FC1F7FE2B880F911D9695879597F989
:103C4000089597F99F6780E870E060E008959FEF1E
:103C500080EC089500240A94161617061806090623
:103C6000089500240A9412161306140605060895F2
:103C7000092E0394000C11F4882352F0BB0F40F47A
:103C8000BF2B11F460FF04C06F5F7F4F8F4F9F4FBA
:103C9000089557FD9058440F551F59F05F3F71F03C
:103CA0004795880F97FB991F61F09F3F79F08795A3
:103CB0000895121613061406551FF2CF4695F1DF2C
:103CC00008C0161617061806991FF1CF86957105BC
:103CD000610508940895E894BB2766277727CB01F0
:103CE00097F90895F999FECF92BD81BDF89A992769
:103CF00080B50895262FF999FECF1FBA92BD81BDD8
:103D000020BD0FB6F894FA9AF99A0FBE019608955D
:103D10002F923F924F925F926F927F928F929F92DB
:103D2000AF92BF92CF92DF92EF92FF920F931F93C9
:103D3000CF93DF93CDB7DEB7CA1BDB0B0FB6F8947A
:103D4000DEBF0FBECDBF09942A88398848885F84BA
:103D50006E847D848C849B84AA84B984C884DF802B
:103D6000EE80FD800C811B81AA81B981CE0FD11D0F
:103D70000FB6F894DEBF0FBECDBFED0108955058C9
:103D8000BB27AA270E94D71E0C94381E0E942A1E09
:103D900038F00E94311E20F039F49F3F19F426F4C8
:103DA0000C94271E0EF4E095E7FB0C94211EE92FDE
:103DB0000E94491E58F3BA176207730784079507D4
:103DC00020F079F4A6F50C946B1E0EF4E0950B2E02
:103DD000BA2FA02D0B01B90190010C01CA01A0015D
:103DE0001124FF27591B99F0593F50F4503E68F1B8
:103DF0001A16F040A22F232F342F4427585FF3CFF9
:103E0000469537952795A795F0405395C9F77EF4C9
:103E10001F16BA0B620B730B840BBAF09150A1F012
:103E2000FF0FBB1F661F771F881FC2F70EC0BA0F98
:103E3000621F731F841F48F4879577956795B79520
:103E4000F7959E3F08F0B0CF9395880F08F099271B
:103E5000EE0F9795879508950E94401F0C94381E89
:103E60000E94311E58F00E942A1E40F029F45F3F44
:103E700029F00C94211E51110C946C1E0C94271ED9
:103E80000E94491E68F39923B1F3552391F3951BC2
:103E9000550BBB27AA2762177307840738F09F5F6B
:103EA0005F4F220F331F441FAA1FA9F335D00E2ED8
:103EB0003AF0E0E832D091505040E695001CCAF745
:103EC0002BD0FE2F29D0660F771F881FBB1F261708
:103ED00037074807AB07B0E809F0BB0B802DBF01DF
:103EE000FF2793585F4F3AF09E3F510578F00C94AE
:103EF000211E0C946C1E5F3FE4F3983ED4F386952C
:103F000077956795B795F7959F5FC9F7880F911DCE
:103F10009695879597F90895E1E0660F771F881FBA
:103F2000BB1F621773078407BA0720F0621B730B6D
:103F3000840BBA0BEE1F88F7E09508950E94A51F29
:103F40006894B1110C946C1E08950E94511E88F063
:103F50009F5798F0B92F9927B751B0F0E1F0660F4D
:103F6000771F881F991F1AF0BA95C9F714C0B1308E
:103F700091F00E946B1EB1E008950C946B1E672FA8
:103F8000782F8827B85F39F0B93FCCF386957795BD
:103F90006795B395D9F73EF49095809570956195A6
:103FA0007F4F8F4F9F4F08950E94901D08F48FEF11
:103FB000089516F00C9429200C94271E68940C94F4
:103FC000211E0E94511EA8F39923C1F3AEF3DF9383
:103FD000CF931F930F93FF92C92FDD2788232AF0D9
:103FE0002197660F771F881FDAF720E030E040E85E
:103FF0005FEB9FE3883920F0803E38F021968F7781
:104000000E94C01EE8E6F0E004C00E94C01EE5E980
:10401000F0E00E9437208B01BE01EC01FB2E6F57B0
:1040200071097595771F880B990B0E94551D28E122
:1040300032E741E35FE30E94C71DAF2D9801AE0157
:10404000FF900F911F91CF91DF910E94D71E0C948A
:10405000381E9F3F31F0915020F4879577956795F2
:10406000B795880F911D9695879597F90895DF93D9
:10407000CF931F930F93FF92EF92DF927B018C01FE
:10408000689406C0DA2EEF010E94C71DFE01E89475
:10409000A5912591359145915591A6F3EF010E9487
:1040A000D71EFE019701A801DA9469F7DF90EF901F
:1040B000FF900F911F91CF91DF910895991B79E0A7
:1040C00004C0991F961708F0961B881F7A95C9F7A8
:1040D0008095089597FB072E16F4009407D077FD7E
:1040E00009D00E949D2007FC05D03EF49095819553
:1040F0009F4F0895709561957F4F0895052E97FB0A
:104100001EF400940E94952057FD07D00E94B12014
:1041100007FC03D04EF40C949520509540953095B3
:1041200021953F4F4F4F5F4F089590958095709523
:1041300061957F4F8F4F9F4F0895AA1BBB1B51E185
:1041400007C0AA1FBB1FA617B70710F0A61BB70B07
:10415000881F991F5A95A9F780959095BC01CD01AC
:104160000895A1E21A2EAA1BBB1BFD010DC0AA1FB8
:10417000BB1FEE1FFF1FA217B307E407F50720F0D0
:10418000A21BB30BE40BF50B661F771F881F991F4B
:104190001A9469F760957095809590959B01AC0194
:1041A000BD01CF010895EE0FFF1F0590F491E02DA2
:1041B00009940F931F93CF93DF938230910510F4EE
:1041C00082E090E0E091AC04F091AD0430E020E0BA
:1041D000B0E0A0E0309799F42115310509F44AC008
:1041E000281B390B24303105D8F58A819B81611554
:1041F000710589F1FB0193838283FE0111C0408127
:1042000051810281138148175907E0F04817590777
:1042100099F4109761F012960C93129713961C93D1
:104220003296CF01DF91CF911F910F9108950093A6
:10423000AC041093AD04F4CF2115310551F04217B1
:10424000530738F0A901DB019A01BD01DF01F80134
:10425000C1CFEF01F9CF9093AD048093AC04CDCFE3
:10426000FE01E20FF31F81939193225031093983AC
:104270002883D7CF2091AA043091AB04232B41F49B
:1042800020918801309189013093AB042093AA04D6
:1042900020918601309187012115310541F42DB718
:1042A0003EB740918A0150918B01241B350BE09160
:1042B000AA04F091AB04E217F307A0F42E1B3F0B06
:1042C0002817390778F0AC014E5F5F4F2417350788
:1042D00048F04E0F5F1F5093AB044093AA048193A4
:1042E00091939FCFF0E0E0E09CCFCF93DF930097D6
:1042F000E9F0FC01329713821282A091AC04B091D4
:10430000AD04ED0130E020E01097A1F4208131816F
:10431000820F931F2091AA043091AB04281739070C
:1043200009F061C0F093AB04E093AA04DF91CF9150
:104330000895EA01CE17DF07E8F54A815B819E0107
:1043400041155105B1F7E901FB83EA834991599180
:10435000C40FD51FEC17FD0761F48081918102968F
:10436000840F951FE90199838883828193819B83C0
:104370008A83F0E0E0E012968D919C91139700976C
:10438000B9F52D913C911197CD010296820F931FA3
:104390002091AA043091AB042817390739F63097D9
:1043A00051F51092AD041092AC04B093AB04A093FD
:1043B000AA04BCCFD383C28340815181840F951F4F
:1043C000C817D90761F44E5F5F4F88819981480F04
:1043D000591F518340838A819B8193838283211556
:1043E000310509F0B0CFF093AD04E093AC049ECF5B
:1043F000FD01DC01C0CF13821282D7CFB0E0A0E074
:10440000E4E0F2E20C948A1E8C01009751F4CB0197
:104410000E94D9208C01C801CDB7DEB7E0E10C9431
:10442000A61EFC01E60FF71F9C0122503109E2177E
:10443000F30708F49DC0D901CD91DC911197C617FF
:10444000D70798F0C530D10530F3CE010497861711
:10445000970708F3C61BD70B2297C193D1936D938F
:104460007C93CF010E947521D6CF5B01AC1ABD0AA7
:104470004C018C0E9D1EA091AC04B091AD04512C4A
:10448000412CF12CE12C109731F58091AA049091E8
:10449000AB048815990509F05CC04616570608F06C
:1044A00058C08091860190918701009741F48DB7A3
:1044B0009EB740918A0150918B01841B950BE817A0
:1044C000F90708F055C0F093AB04E093AA04F90192
:1044D00071836083A0CF8D919C91119712966C90FF
:1044E000129713967C901397A815B90559F56C018E
:1044F00042E0C40ED11CCA14DB0420F1AC014A19FD
:104500005B09DA011296159780F0628273825183FB
:104510004083D9016D937C93E114F10471F0D701CC
:104520001396FC93EE93129776CF22968C0F9D1FD5
:10453000F90191838083F301EFCFF093AD04E09311
:10454000AC0469CF4816590608F42C017D01D3014B
:104550009ACFCB010E94D9207C01009749F0AE018F
:10456000B8010E94BB22C8010E947521870153CF68
:1045700010E000E050CFFB01DC0102C001900D9281
:1045800041505040D8F70895FC018191861721F0E1
:104590008823D9F7992708953197CF010895FB0112
:1045A000DC018D91019080190110D9F3990B0895C8
:1045B000FB01DC0101900D920020E1F70895FB0161
:1045C00051915523A9F0BF01DC014D9145174111CF
:1045D000E1F759F4CD010190002049F04D914015CB
:1045E0004111C9F3FB014111EFCF81E090E0019748
:1045F000089511E0C2E8D1E004C0FE010E94D3207A
:0C4600002196C338D107C9F7F894FFCF0A
:10460C00224E5445204750532120202041545445DC
:10461C0028000000000000002740410000000000BE
:10462C002600000000000000250000000000000033
:10463C002400000000000000230000000000000027
:10464C00220000000000000021000000000000001B
:10465C00103E2B820002002A01FFFFFFFFFFA20089
:10466C00000000000000800000000000000040007E
:10467C0000000000230001000000000000004000CA
:10468C000000000000000000AE04800004081030A0
:10469C004050041040000000009F02FF012C020754
:1046AC00035D023B024F02000000001404FF01A94D
:1046BC0004130470048804FB03303E00313E0032C6
:1046CC003E00333E00343E00353E00363E00203284
:1046DC003000352E342064752033302F31312F3299
:1046EC003031390044696D616E636865004C756EDC
:1046FC006469004D61726469004D65726372656432
:10470C0069004A657564690056656E647265646912
:10471C000053616D656469006A616E76696572004B
:10472C0066657672696572006D617273006176728E
:10473C00696C006D6169006A75696E006A75696CF7
:10474C006C657400616F75740073657074656D626F
:10475C007265006F63746F627265006E6F76656D63
:10476C0062726500646563656D62726500456E74A6
:10477C0065722073657474696E67206D6F64652053
:10478C006661696C0D0A00456E7465722073657400
:10479C0074696E67206D6F646520737563636573F0
:1047AC0073200D0A00736574207261746520737533
:1047BC00636365737321210D0A00456E7465722065
:1047CC004E6F726D616C204D6F6465204661696C33
:1047DC0021210D0A00456E746572204E6F726D6159
:1047EC006C204D6F64652053756363657373212171
:0447FC000D0A0000A2
:00000001FF
